 declcls003

 Timestamp is ac47e340 (reproducible build file hash)

 Preferred load address is 0000000180000000

 Start         Length     Name                   Class
 0001:00000000 00002be0H .text$mn                CODE
 0001:00002be0 00000036H .text$mn$00             CODE
 0001:00002c16 00000092H .text$x                 CODE
 0002:00000000 00000198H .idata$5                DATA
 0002:00000198 00000038H .00cfg                  DATA
 0002:000001d0 00000008H .CRT$XCA                DATA
 0002:000001d8 00000008H .CRT$XCZ                DATA
 0002:000001e0 00000008H .CRT$XIA                DATA
 0002:000001e8 00000008H .CRT$XIC                DATA
 0002:000001f0 00000008H .CRT$XIZ                DATA
 0002:000001f8 00000008H .CRT$XLA                DATA
 0002:00000200 00000008H .CRT$XLZ                DATA
 0002:00000208 00000008H .CRT$XPA                DATA
 0002:00000210 00000008H .CRT$XPZ                DATA
 0002:00000218 00000008H .CRT$XTA                DATA
 0002:00000220 00000010H .CRT$XTZ                DATA
 0002:00000228 00000000H .gehcont$y              DATA
 0002:00000228 00000000H .gfids$y                DATA
 0002:00000230 00001bd0H .rdata                  DATA
 0002:00001e00 00000000H .rdata$CastGuardVftablesA DATA
 0002:00001e00 00000000H .rdata$CastGuardVftablesC DATA
 0002:00001e00 00000028H .rdata$T                DATA
 0002:00001e28 000000b0H .rdata$voltmd           DATA
 0002:00001ed8 00000318H .rdata$zzzdbg           DATA
 0002:000021f0 00000008H .rtc$IAA                DATA
 0002:000021f8 00000008H .rtc$IZZ                DATA
 0002:00002200 00000008H .rtc$TAA                DATA
 0002:00002208 00000008H .rtc$TZZ                DATA
 0002:00002210 00000004H .tls                    DATA
 0002:00002214 00000004H .tls$                   DATA
 0002:00002218 00000008H .tls$ZZZ                DATA
 0002:00002220 000002f0H .xdata                  DATA
 0002:00002510 000003a4H .edata                  DATA
 0002:000028b4 00000064H .idata$2                DATA
 0002:00002918 00000018H .idata$3                DATA
 0002:00002930 00000198H .idata$4                DATA
 0002:00002ac8 0000041eH .idata$6                DATA
 0003:00000000 000000e0H .data                   DATA
 0003:000000e0 0001b238H .bss                    DATA
 0004:00000000 00000378H .pdata                  DATA

  Address         Publics by Value              Rva+Base               Lib:Object

 0000:00000000       __AbsoluteZero             0000000000000000     <absolute>
 0000:00000000       ___safe_se_handler_count   0000000000000000     <absolute>
 0000:00000000       ___safe_se_handler_table   0000000000000000     <absolute>
 0000:00000000       __arm64x_extra_rfe_table   0000000000000000     <absolute>
 0000:00000000       __arm64x_extra_rfe_table_size 0000000000000000     <absolute>
 0000:00000000       __arm64x_native_entrypoint 0000000000000000     <absolute>
 0000:00000000       __arm64x_redirection_metadata 0000000000000000     <absolute>
 0000:00000000       __arm64x_redirection_metadata_count 0000000000000000     <absolute>
 0000:00000000       __dynamic_value_reloc_table 0000000000000000     <absolute>
 0000:00000000       __enclave_config           0000000000000000     <absolute>
 0000:00000000       __guard_check_icall_a64n_fptr 0000000000000000     <absolute>
 0000:00000000       __guard_eh_cont_count      0000000000000000     <absolute>
 0000:00000000       __guard_eh_cont_table      0000000000000000     <absolute>
 0000:00000000       __guard_fids_count         0000000000000000     <absolute>
 0000:00000000       __guard_fids_table         0000000000000000     <absolute>
 0000:00000000       __guard_iat_count          0000000000000000     <absolute>
 0000:00000000       __guard_iat_table          0000000000000000     <absolute>
 0000:00000000       __guard_longjmp_count      0000000000000000     <absolute>
 0000:00000000       __guard_longjmp_table      0000000000000000     <absolute>
 0000:00000000       __hybrid_auxiliary_iat     0000000000000000     <absolute>
 0000:00000000       __hybrid_auxiliary_iat_copy 0000000000000000     <absolute>
 0000:00000000       __hybrid_code_map          0000000000000000     <absolute>
 0000:00000000       __hybrid_code_map_count    0000000000000000     <absolute>
 0000:00000000       __x64_code_ranges_to_entry_points 0000000000000000     <absolute>
 0000:00000000       __x64_code_ranges_to_entry_points_count 0000000000000000     <absolute>
 0000:00000100       __guard_flags              0000000000000100     <absolute>
 0000:00000000       __ImageBase                0000000180000000     <linker-defined>
 0001:00000000       ?NewObject@JNIEnv_@@QEAAPEAV_jobject@@PEAV_jclass@@PEAU_jmethodID@@ZZ 0000000180001000 f i libdeclcls003.obj
 0001:00000024       ?TranslateError@@YAPEBDW4jvmtiError@@@Z 0000000180001024 f   libdeclcls003.obj
 0001:000002dc       ?nsk_jni_check_exception@@YAHPEAUJNIEnv_@@QEBDH@Z 00000001800012dc f   libdeclcls003.obj
 0001:00000420       ?nsk_jni_lverify@@YAHHPEAUJNIEnv_@@HQEBDH1ZZ 0000000180001420 f   libdeclcls003.obj
 0001:000004c0       Agent_Initialize           00000001800014c0 f   libdeclcls003.obj
 0001:00000530       Agent_OnAttach             0000000180001530 f   libdeclcls003.obj
 0001:00000530       Agent_OnLoad               0000000180001530 f   libdeclcls003.obj
 0001:00000538       Java_nsk_jvmti_GetMethodDeclaringClass_declcls003_check 0000000180001538 f   libdeclcls003.obj
 0001:00000698       Java_nsk_jvmti_unit_FollowReferences_FollowRefObjects_addRefToVerify 0000000180001698 f   libdeclcls003.obj
 0001:00000854       Java_nsk_jvmti_unit_FollowReferences_FollowRefObjects_getTag 0000000180001854 f   libdeclcls003.obj
 0001:00000910       Java_nsk_jvmti_unit_FollowReferences_FollowRefObjects_resetRefsToVerify 0000000180001910 f   libdeclcls003.obj
 0001:00000918       Java_nsk_jvmti_unit_FollowReferences_FollowRefObjects_resetTags 0000000180001918 f   libdeclcls003.obj
 0001:0000095c       Java_nsk_jvmti_unit_FollowReferences_FollowRefObjects_setTag 000000018000195c f   libdeclcls003.obj
 0001:00000ba8       Java_nsk_share_jvmti_ArgumentHandler_getAgentOptionsString 0000000180001ba8 f   libdeclcls003.obj
 0001:00000c54       Java_nsk_share_jvmti_DebugeeClass_checkStatus 0000000180001c54 f   libdeclcls003.obj
 0001:00000cdc       Java_nsk_share_jvmti_DebugeeClass_resetAgentData 0000000180001cdc f   libdeclcls003.obj
 0001:00000d3c       Java_nsk_share_jvmti_RedefineAgent_agentStatus 0000000180001d3c f   libdeclcls003.obj
 0001:00000d48       Java_nsk_share_jvmti_RedefineAgent_isRedefined 0000000180001d48 f   libdeclcls003.obj
 0001:00000d54       Java_nsk_share_jvmti_RedefineAgent_redefineAttempted 0000000180001d54 f   libdeclcls003.obj
 0001:00000d60       MA_checkStatus             0000000180001d60 f   libdeclcls003.obj
 0001:00000e04       __local_stdio_printf_options 0000000180001e04 f i libdeclcls003.obj
 0001:00000fd4       do_check                   0000000180001fd4 f   libdeclcls003.obj
 0001:0000115c       exitOnError                000000018000215c f   libdeclcls003.obj
 0001:00001210       fprintf                    0000000180002210 f i libdeclcls003.obj
 0001:00001254       nsk_jvmti_lverify          0000000180002254 f   libdeclcls003.obj
 0001:00001344       nsk_jvmti_resetAgentData   0000000180002344 f   libdeclcls003.obj
 0001:000013b8       nsk_lcomplain              00000001800023b8 f   libdeclcls003.obj
 0001:000013d8       nsk_ldisplay               00000001800023d8 f   libdeclcls003.obj
 0001:000013f8       nsk_ltrace                 00000001800023f8 f   libdeclcls003.obj
 0001:00001418       nsk_lvcomplain             0000000180002418 f   libdeclcls003.obj
 0001:000015d0       nsk_lvdisplay              00000001800025d0 f   libdeclcls003.obj
 0001:0000161c       nsk_lverify                000000018000261c f   libdeclcls003.obj
 0001:00001678       nsk_lvtrace                0000000180002678 f   libdeclcls003.obj
 0001:000016d8       nsk_printf                 00000001800026d8 f   libdeclcls003.obj
 0001:00001700       nsk_vprintf                0000000180002700 f   libdeclcls003.obj
 0001:000017b4       printf                     00000001800027b4 f i libdeclcls003.obj
 0001:00001cb4       __raise_securityfailure    0000000180002cb4 f   MSVCRT:gs_report.obj
 0001:00001ce8       __report_gsfailure         0000000180002ce8 f   MSVCRT:gs_report.obj
 0001:00001f28       __GSHandlerCheck           0000000180002f28 f   MSVCRT:gshandler.obj
 0001:00001f48       __GSHandlerCheckCommon     0000000180002f48 f   MSVCRT:gshandler.obj
 0001:00001fc0       __security_check_cookie    0000000180002fc0 f   MSVCRT:amdsecgs.obj
 0001:00002300       _DllMainCRTStartup         0000000180003300 f   MSVCRT:dll_dllmain.obj
 0001:00002340       __scrt_acquire_startup_lock 0000000180003340 f   MSVCRT:utility.obj
 0001:0000237c       __scrt_dllmain_after_initialize_c 000000018000337c f   MSVCRT:utility.obj
 0001:000023b0       __scrt_dllmain_before_initialize_c 00000001800033b0 f   MSVCRT:utility.obj
 0001:000023c8       __scrt_dllmain_crt_thread_attach 00000001800033c8 f   MSVCRT:utility.obj
 0001:000023f0       __scrt_dllmain_crt_thread_detach 00000001800033f0 f   MSVCRT:utility.obj
 0001:00002408       __scrt_dllmain_exception_filter 0000000180003408 f   MSVCRT:utility.obj
 0001:00002468       __scrt_dllmain_uninitialize_c 0000000180003468 f   MSVCRT:utility.obj
 0001:00002498       __scrt_dllmain_uninitialize_critical 0000000180003498 f   MSVCRT:utility.obj
 0001:000024ac       __scrt_initialize_crt      00000001800034ac f   MSVCRT:utility.obj
 0001:000024f8       __scrt_initialize_onexit_tables 00000001800034f8 f   MSVCRT:utility.obj
 0001:00002584       __scrt_is_nonwritable_in_current_image 0000000180003584 f   MSVCRT:utility.obj
 0001:0000261c       __scrt_release_startup_lock 000000018000361c f   MSVCRT:utility.obj
 0001:00002640       __scrt_uninitialize_crt    0000000180003640 f   MSVCRT:utility.obj
 0001:0000266c       _onexit                    000000018000366c f   MSVCRT:utility.obj
 0001:000026a8       atexit                     00000001800036a8 f   MSVCRT:utility.obj
 0001:000026c0       __crt_debugger_hook        00000001800036c0 f   MSVCRT:utility_desktop.obj
 0001:000026c8       __scrt_fastfail            00000001800036c8 f   MSVCRT:utility_desktop.obj
 0001:00002814       _guard_check_icall_nop     0000000180003814 f i MSVCRT:guard_support.obj
 0001:00002818       __security_init_cookie     0000000180003818 f   MSVCRT:gs_support.obj
 0001:000028c4       DllMain                    00000001800038c4 f   MSVCRT:dll_dllmain_stub.obj
 0001:000028e8       ?__scrt_initialize_type_info@@YAXXZ 00000001800038e8 f   MSVCRT:tncleanup.obj
 0001:000028f8       ?__scrt_uninitialize_type_info@@YAXXZ 00000001800038f8 f   MSVCRT:tncleanup.obj
 0001:00002904       __local_stdio_scanf_options 0000000180003904 f i MSVCRT:default_local_stdio_options.obj
 0001:0000290c       __scrt_initialize_default_local_stdio_options 000000018000390c f   MSVCRT:default_local_stdio_options.obj
 0001:00002928       __scrt_get_dyn_tls_init_callback 0000000180003928 f   MSVCRT:dyn_tls_init.obj
 0001:00002930       _RTC_Initialize            0000000180003930 f   MSVCRT:initsect.obj
 0001:0000296c       _RTC_Terminate             000000018000396c f   MSVCRT:initsect.obj
 0001:000029a8       __isa_available_init       00000001800039a8 f   MSVCRT:cpu_disp.obj
 0001:00002b54       _get_startup_argv_mode     0000000180003b54 f   MSVCRT:argv_mode.obj
 0001:00002b5c       __scrt_is_ucrt_dll_in_use  0000000180003b5c f   MSVCRT:ucrt_detection.obj
 0001:00002b70       memcpy                     0000000180003b70 f   vcruntime:VCRUNTIME140.dll
 0001:00002b76       memset                     0000000180003b76 f   vcruntime:VCRUNTIME140.dll
 0001:00002b7c       strchr                     0000000180003b7c f   vcruntime:VCRUNTIME140.dll
 0001:00002b82       __C_specific_handler       0000000180003b82 f   vcruntime:VCRUNTIME140.dll
 0001:00002b88       __std_type_info_destroy_list 0000000180003b88 f   vcruntime:VCRUNTIME140.dll
 0001:00002b8e       strcmp                     0000000180003b8e f   ucrt:api-ms-win-crt-string-l1-1-0.dll
 0001:00002b94       strlen                     0000000180003b94 f   ucrt:api-ms-win-crt-string-l1-1-0.dll
 0001:00002b9a       _initterm                  0000000180003b9a f   ucrt:api-ms-win-crt-runtime-l1-1-0.dll
 0001:00002ba0       _initterm_e                0000000180003ba0 f   ucrt:api-ms-win-crt-runtime-l1-1-0.dll
 0001:00002ba6       _seh_filter_dll            0000000180003ba6 f   ucrt:api-ms-win-crt-runtime-l1-1-0.dll
 0001:00002bac       _configure_narrow_argv     0000000180003bac f   ucrt:api-ms-win-crt-runtime-l1-1-0.dll
 0001:00002bb2       _initialize_narrow_environment 0000000180003bb2 f   ucrt:api-ms-win-crt-runtime-l1-1-0.dll
 0001:00002bb8       _initialize_onexit_table   0000000180003bb8 f   ucrt:api-ms-win-crt-runtime-l1-1-0.dll
 0001:00002bbe       _register_onexit_function  0000000180003bbe f   ucrt:api-ms-win-crt-runtime-l1-1-0.dll
 0001:00002bc4       _execute_onexit_table      0000000180003bc4 f   ucrt:api-ms-win-crt-runtime-l1-1-0.dll
 0001:00002bca       _crt_atexit                0000000180003bca f   ucrt:api-ms-win-crt-runtime-l1-1-0.dll
 0001:00002bd0       _cexit                     0000000180003bd0 f   ucrt:api-ms-win-crt-runtime-l1-1-0.dll
 0001:00002bd8       __acrt_initialize          0000000180003bd8 f   MSVCRT:ucrt_stubs.obj
 0001:00002bd8       __acrt_thread_attach       0000000180003bd8 f   MSVCRT:ucrt_stubs.obj
 0001:00002bd8       __acrt_thread_detach       0000000180003bd8 f   MSVCRT:ucrt_stubs.obj
 0001:00002bd8       __acrt_uninitialize        0000000180003bd8 f   MSVCRT:ucrt_stubs.obj
 0001:00002bd8       __acrt_uninitialize_critical 0000000180003bd8 f   MSVCRT:ucrt_stubs.obj
 0001:00002bd8       __scrt_stub_for_acrt_initialize 0000000180003bd8 f   MSVCRT:ucrt_stubs.obj
 0001:00002bd8       __scrt_stub_for_acrt_thread_attach 0000000180003bd8 f   MSVCRT:ucrt_stubs.obj
 0001:00002bd8       __scrt_stub_for_acrt_thread_detach 0000000180003bd8 f   MSVCRT:ucrt_stubs.obj
 0001:00002bd8       __scrt_stub_for_acrt_uninitialize 0000000180003bd8 f   MSVCRT:ucrt_stubs.obj
 0001:00002bd8       __scrt_stub_for_acrt_uninitialize_critical 0000000180003bd8 f   MSVCRT:ucrt_stubs.obj
 0001:00002bd8       __vcrt_initialize          0000000180003bd8 f   MSVCRT:ucrt_stubs.obj
 0001:00002bd8       __vcrt_thread_attach       0000000180003bd8 f   MSVCRT:ucrt_stubs.obj
 0001:00002bd8       __vcrt_thread_detach       0000000180003bd8 f   MSVCRT:ucrt_stubs.obj
 0001:00002bd8       __vcrt_uninitialize        0000000180003bd8 f   MSVCRT:ucrt_stubs.obj
 0001:00002bd8       __vcrt_uninitialize_critical 0000000180003bd8 f   MSVCRT:ucrt_stubs.obj
 0001:00002bdc       __scrt_stub_for_is_c_termination_complete 0000000180003bdc f   MSVCRT:ucrt_stubs.obj
 0001:00002bdc       _is_c_termination_complete 0000000180003bdc f   MSVCRT:ucrt_stubs.obj
 0001:00002bf0       _guard_dispatch_icall_nop  0000000180003bf0 f   MSVCRT:guard_dispatch.obj
 0001:00002c10       _guard_xfg_dispatch_icall_nop 0000000180003c10 f   MSVCRT:guard_xfg_dispatch.obj
 0002:00000000       __imp_RtlCaptureContext    0000000180004000     kernel32:KERNEL32.dll
 0002:00000008       __imp_RtlLookupFunctionEntry 0000000180004008     kernel32:KERNEL32.dll
 0002:00000010       __imp_RtlVirtualUnwind     0000000180004010     kernel32:KERNEL32.dll
 0002:00000018       __imp_UnhandledExceptionFilter 0000000180004018     kernel32:KERNEL32.dll
 0002:00000020       __imp_SetUnhandledExceptionFilter 0000000180004020     kernel32:KERNEL32.dll
 0002:00000028       __imp_GetCurrentProcess    0000000180004028     kernel32:KERNEL32.dll
 0002:00000030       __imp_TerminateProcess     0000000180004030     kernel32:KERNEL32.dll
 0002:00000038       __imp_IsProcessorFeaturePresent 0000000180004038     kernel32:KERNEL32.dll
 0002:00000040       __imp_CloseHandle          0000000180004040     kernel32:KERNEL32.dll
 0002:00000048       __imp_InitializeCriticalSectionAndSpinCount 0000000180004048     kernel32:KERNEL32.dll
 0002:00000050       __imp_DeleteCriticalSection 0000000180004050     kernel32:KERNEL32.dll
 0002:00000058       __imp_CreateEventW         0000000180004058     kernel32:KERNEL32.dll
 0002:00000060       __imp_GetModuleHandleW     0000000180004060     kernel32:KERNEL32.dll
 0002:00000068       __imp_GetProcAddress       0000000180004068     kernel32:KERNEL32.dll
 0002:00000070       __imp_IsDebuggerPresent    0000000180004070     kernel32:KERNEL32.dll
 0002:00000078       __imp_QueryPerformanceCounter 0000000180004078     kernel32:KERNEL32.dll
 0002:00000080       __imp_GetCurrentProcessId  0000000180004080     kernel32:KERNEL32.dll
 0002:00000088       __imp_GetCurrentThreadId   0000000180004088     kernel32:KERNEL32.dll
 0002:00000090       __imp_GetSystemTimeAsFileTime 0000000180004090     kernel32:KERNEL32.dll
 0002:00000098       __imp_DisableThreadLibraryCalls 0000000180004098     kernel32:KERNEL32.dll
 0002:000000a0       __imp_InitializeSListHead  00000001800040a0     kernel32:KERNEL32.dll
 0002:000000a8       \177KERNEL32_NULL_THUNK_DATA 00000001800040a8     kernel32:KERNEL32.dll
 0002:000000b0       __imp_memcpy               00000001800040b0     vcruntime:VCRUNTIME140.dll
 0002:000000b8       __imp_memset               00000001800040b8     vcruntime:VCRUNTIME140.dll
 0002:000000c0       __imp_strchr               00000001800040c0     vcruntime:VCRUNTIME140.dll
 0002:000000c8       __imp___C_specific_handler 00000001800040c8     vcruntime:VCRUNTIME140.dll
 0002:000000d0       __imp___std_type_info_destroy_list 00000001800040d0     vcruntime:VCRUNTIME140.dll
 0002:000000d8       \177VCRUNTIME140_NULL_THUNK_DATA 00000001800040d8     vcruntime:VCRUNTIME140.dll
 0002:000000e0       __imp__errno               00000001800040e0     ucrt:api-ms-win-crt-runtime-l1-1-0.dll
 0002:000000e8       __imp_exit                 00000001800040e8     ucrt:api-ms-win-crt-runtime-l1-1-0.dll
 0002:000000f0       __imp__cexit               00000001800040f0     ucrt:api-ms-win-crt-runtime-l1-1-0.dll
 0002:000000f8       __imp__crt_atexit          00000001800040f8     ucrt:api-ms-win-crt-runtime-l1-1-0.dll
 0002:00000100       __imp__execute_onexit_table 0000000180004100     ucrt:api-ms-win-crt-runtime-l1-1-0.dll
 0002:00000108       __imp__register_onexit_function 0000000180004108     ucrt:api-ms-win-crt-runtime-l1-1-0.dll
 0002:00000110       __imp__initialize_onexit_table 0000000180004110     ucrt:api-ms-win-crt-runtime-l1-1-0.dll
 0002:00000118       __imp__initialize_narrow_environment 0000000180004118     ucrt:api-ms-win-crt-runtime-l1-1-0.dll
 0002:00000120       __imp__configure_narrow_argv 0000000180004120     ucrt:api-ms-win-crt-runtime-l1-1-0.dll
 0002:00000128       __imp__seh_filter_dll      0000000180004128     ucrt:api-ms-win-crt-runtime-l1-1-0.dll
 0002:00000130       __imp__initterm_e          0000000180004130     ucrt:api-ms-win-crt-runtime-l1-1-0.dll
 0002:00000138       __imp__initterm            0000000180004138     ucrt:api-ms-win-crt-runtime-l1-1-0.dll
 0002:00000140       \177api-ms-win-crt-runtime-l1-1-0_NULL_THUNK_DATA 0000000180004140     ucrt:api-ms-win-crt-runtime-l1-1-0.dll
 0002:00000148       __imp___acrt_iob_func      0000000180004148     ucrt:api-ms-win-crt-stdio-l1-1-0.dll
 0002:00000150       __imp_fflush               0000000180004150     ucrt:api-ms-win-crt-stdio-l1-1-0.dll
 0002:00000158       __imp___stdio_common_vsprintf 0000000180004158     ucrt:api-ms-win-crt-stdio-l1-1-0.dll
 0002:00000160       __imp___stdio_common_vfprintf 0000000180004160     ucrt:api-ms-win-crt-stdio-l1-1-0.dll
 0002:00000168       \177api-ms-win-crt-stdio-l1-1-0_NULL_THUNK_DATA 0000000180004168     ucrt:api-ms-win-crt-stdio-l1-1-0.dll
 0002:00000170       __imp_strcmp               0000000180004170     ucrt:api-ms-win-crt-string-l1-1-0.dll
 0002:00000178       __imp__strdup              0000000180004178     ucrt:api-ms-win-crt-string-l1-1-0.dll
 0002:00000178       __imp_strdup               0000000180004178     ucrt:api-ms-win-crt-string-l1-1-0.dll
 0002:00000180       __imp_strlen               0000000180004180     ucrt:api-ms-win-crt-string-l1-1-0.dll
 0002:00000188       __imp_strncpy              0000000180004188     ucrt:api-ms-win-crt-string-l1-1-0.dll
 0002:00000190       \177api-ms-win-crt-string-l1-1-0_NULL_THUNK_DATA 0000000180004190     ucrt:api-ms-win-crt-string-l1-1-0.dll
 0002:00000198       __guard_check_icall_fptr   0000000180004198     MSVCRT:guard_support.obj
 0002:000001a0       __guard_xfg_check_icall_fptr 00000001800041a0     MSVCRT:guard_support.obj
 0002:000001a8       __guard_dispatch_icall_fptr 00000001800041a8     MSVCRT:guard_support.obj
 0002:000001b0       __guard_xfg_dispatch_icall_fptr 00000001800041b0     MSVCRT:guard_support.obj
 0002:000001b8       __guard_xfg_table_dispatch_icall_fptr 00000001800041b8     MSVCRT:guard_support.obj
 0002:000001c0       __castguard_check_failure_os_handled_fptr 00000001800041c0     MSVCRT:guard_support.obj
 0002:000001c8       __guard_memcpy_fptr        00000001800041c8     vcruntime:softmemtag.obj
 0002:000001d0       __xc_a                     00000001800041d0     MSVCRT:initializers.obj
 0002:000001d8       __xc_z                     00000001800041d8     MSVCRT:initializers.obj
 0002:000001e0       __xi_a                     00000001800041e0     MSVCRT:initializers.obj
 0002:000001f0       __xi_z                     00000001800041f0     MSVCRT:initializers.obj
 0002:000001f8       __xl_a                     00000001800041f8     MSVCRT:tlssup.obj
 0002:00000200       __xl_z                     0000000180004200     MSVCRT:tlssup.obj
 0002:00000208       __xp_a                     0000000180004208     MSVCRT:initializers.obj
 0002:00000210       __xp_z                     0000000180004210     MSVCRT:initializers.obj
 0002:00000218       __xt_a                     0000000180004218     MSVCRT:initializers.obj
 0002:00000220       __xt_z                     0000000180004220     MSVCRT:initializers.obj
 0002:00000230       g_refKindStr               0000000180004230     libdeclcls003.obj
 0002:000003e0       ??_C@_09BPLDFGCI@unknown_0@ 00000001800043e0     libdeclcls003.obj
 0002:000003f0       ??_C@_0BL@FPNMECJD@JVMTI_HEAP_REFERENCE_CLASS@ 00000001800043f0     libdeclcls003.obj
 0002:00000410       ??_C@_0BL@FKGKKLNM@JVMTI_HEAP_REFERENCE_FIELD@ 0000000180004410     libdeclcls003.obj
 0002:00000430       ??_C@_0CD@CAEHCFJF@JVMTI_HEAP_REFERENCE_ARRAY_ELEM@ 0000000180004430     libdeclcls003.obj
 0002:00000458       ??_C@_0CC@DNEBMCNK@JVMTI_HEAP_REFERENCE_CLASS_LOAD@ 0000000180004458     libdeclcls003.obj
 0002:00000480       ??_C@_0BN@CJMIPEBB@JVMTI_HEAP_REFERENCE_SIGNERS@ 0000000180004480     libdeclcls003.obj
 0002:000004a0       ??_C@_0CH@HBOIDPEB@JVMTI_HEAP_REFERENCE_PROTECTION@ 00000001800044a0     libdeclcls003.obj
 0002:000004c8       ??_C@_0BP@MDKGDGKL@JVMTI_HEAP_REFERENCE_INTERFACE@ 00000001800044c8     libdeclcls003.obj
 0002:000004e8       ??_C@_0CC@JJMIHNJH@JVMTI_HEAP_REFERENCE_STATIC_FIE@ 00000001800044e8     libdeclcls003.obj
 0002:00000510       ??_C@_0CD@IDHEEGID@JVMTI_HEAP_REFERENCE_CONSTANT_P@ 0000000180004510     libdeclcls003.obj
 0002:00000538       ??_C@_0CA@EFFCHNG@JVMTI_HEAP_REFERENCE_SUPERCLASS@ 0000000180004538     libdeclcls003.obj
 0002:00000558       ??_C@_0L@PCDFHGCJ@unknown_11@ 0000000180004558     libdeclcls003.obj
 0002:00000568       ??_C@_0L@NJBICFOK@unknown_12@ 0000000180004568     libdeclcls003.obj
 0002:00000578       ??_C@_0L@MAADBEKL@unknown_13@ 0000000180004578     libdeclcls003.obj
 0002:00000588       ??_C@_0L@IPECICGM@unknown_14@ 0000000180004588     libdeclcls003.obj
 0002:00000598       ??_C@_0L@JGFJLDCN@unknown_15@ 0000000180004598     libdeclcls003.obj
 0002:000005a8       ??_C@_0L@LNHEOAOO@unknown_16@ 00000001800045a8     libdeclcls003.obj
 0002:000005b8       ??_C@_0L@KEGPNBKP@unknown_17@ 00000001800045b8     libdeclcls003.obj
 0002:000005c8       ??_C@_0L@CDPHMNGA@unknown_18@ 00000001800045c8     libdeclcls003.obj
 0002:000005d8       ??_C@_0L@DKOMPMCB@unknown_19@ 00000001800045d8     libdeclcls003.obj
 0002:000005e8       ??_C@_0L@OJGIPJDB@unknown_20@ 00000001800045e8     libdeclcls003.obj
 0002:000005f8       ??_C@_0CA@KAOFNDEM@JVMTI_HEAP_REFERENCE_JNI_GLOBAL@ 00000001800045f8     libdeclcls003.obj
 0002:00000618       ??_C@_0CC@HPFAJBK@JVMTI_HEAP_REFERENCE_SYSTEM_CLA@ 0000000180004618     libdeclcls003.obj
 0002:00000640       ??_C@_0BN@FDEGFOHC@JVMTI_HEAP_REFERENCE_MONITOR@ 0000000180004640     libdeclcls003.obj
 0002:00000660       ??_C@_0CB@HKIBCMAJ@JVMTI_HEAP_REFERENCE_STACK_LOCA@ 0000000180004660     libdeclcls003.obj
 0002:00000688       ??_C@_0BP@EAACMMOE@JVMTI_HEAP_REFERENCE_JNI_LOCAL@ 0000000180004688     libdeclcls003.obj
 0002:000006a8       ??_C@_0BM@IJDEOGOE@JVMTI_HEAP_REFERENCE_THREAD@ 00000001800046a8     libdeclcls003.obj
 0002:000006c8       ??_C@_0BL@EDGPPKC@JVMTI_HEAP_REFERENCE_OTHER@ 00000001800046c8     libdeclcls003.obj
 0002:000006e4       ??_C@_04BCJPDBDA@Code@     00000001800046e4     libdeclcls003.obj
 0002:000006f0       ??_C@_0BA@OCLMCFKC@LineNumberTable@ 00000001800046f0     libdeclcls003.obj
 0002:00000700       ??_C@_0BD@CPAEPILC@LocalVariableTable@ 0000000180004700     libdeclcls003.obj
 0002:00000718       ??_C@_0BH@NMBDNHBD@LocalVariableTypeTable@ 0000000180004718     libdeclcls003.obj
 0002:00000730       ??_C@_0O@HIHEEDNJ@StackMapTable@ 0000000180004730     libdeclcls003.obj
 0002:00000740       ??_C@_0BD@HMGGFBMH@Ljava?1lang?1Object?$DL@ 0000000180004740     libdeclcls003.obj
 0002:00000754       ??_C@_02KCBIMKDL@?$FLB@    0000000180004754     libdeclcls003.obj
 0002:00000758       ??_C@_02LLADPLHK@?$FLC@    0000000180004758     libdeclcls003.obj
 0002:0000075c       ??_C@_02PEECGNLN@?$FLD@    000000018000475c     libdeclcls003.obj
 0002:00000760       ??_C@_02MGHEAPDP@?$FLF@    0000000180004760     libdeclcls003.obj
 0002:00000764       ??_C@_02EBOMBDPA@?$FLI@    0000000180004764     libdeclcls003.obj
 0002:00000768       ??_C@_02GKMBEADD@?$FLJ@    0000000180004768     libdeclcls003.obj
 0002:0000076c       ??_C@_02PBMBOJCL@?$FLS@    000000018000476c     libdeclcls003.obj
 0002:00000770       ??_C@_02CAADFCGC@?$FLZ@    0000000180004770     libdeclcls003.obj
 0002:00000778       ??_C@_0DA@DGENFAKA@?$FLLnsk?1jvmti?1GetMethodDeclaringC@ 0000000180004778     libdeclcls003.obj
 0002:000007a8       ??_C@_0DB@OKPNFOOA@?$FL?$FLLnsk?1jvmti?1GetMethodDeclaring@ 00000001800047a8     libdeclcls003.obj
 0002:000007e0       ??_C@_0L@HCDIAMJG@?9?5?$CFs?0?5?$CFd?3?5@ 00000001800047e0     libdeclcls003.obj
 0002:000007f0       ??_C@_0JI@HLPECLFI@?$CD?5?4?4?4?6?$CD?5ERROR?3?5too?5many?5complai@ 00000001800047f0     libdeclcls003.obj
 0002:00000890       ??_C@_0ED@JNEKCCOB@The?5following?5fake?5exception?5st@ 0000000180004890     libdeclcls003.obj
 0002:000008d8       ??_C@_0CN@FCNMDFBH@nsk?4share?4Fake_Exception_for_RU@ 00000001800048d8     libdeclcls003.obj
 0002:00000908       ??_C@_08PGFFNAEI@?$CI?$CFs?3?$CFd?$CJ?5@ 0000000180004908     libdeclcls003.obj
 0002:00000918       ??_C@_0DP@IENMAEGI@s?2test?2hotspot?2jtreg?2vmTestbase@ 0000000180004918     libdeclcls003.obj
 0002:00000958       ??_C@_0BL@NDJLFFJB@?7at?5nsk_lvcomplain?$CI?$CFs?3?$CFd?$CJ?6@ 0000000180004958     libdeclcls003.obj
 0002:00000978       ??_C@_0BC@JOOKAFKF@?$CD?5ERROR?3?5?$CFs?0?5?$CFd?3?5@ 0000000180004978     libdeclcls003.obj
 0002:00000990       ??_C@_09KJEAHMEH@?$CD?5ERROR?3?5@ 0000000180004990     libdeclcls003.obj
 0002:0000099c       ??_C@_02GPIOPFAK@?$DO?$DO@ 000000018000499c     libdeclcls003.obj
 0002:000009a0       ??_C@_02FODMEDOG@?$DM?$DM@ 00000001800049a0     libdeclcls003.obj
 0002:000009a4       ??_C@_02DJGKEECL@?4?4@     00000001800049a4     libdeclcls003.obj
 0002:000009a8       ??_C@_0O@CJPGJOAF@?9?5?$CFs?0?5?$CFd?3?5?$CFs?5@ 00000001800049a8     libdeclcls003.obj
 0002:000009b8       ??_C@_0CB@IAKPDOIC@?$CD?5?5?5verified?5assertion?5is?5FALSE@ 00000001800049b8     libdeclcls003.obj
 0002:000009e0       ??_C@_0CO@LGONDEPD@stdout?3?5fflush?5failed?5?9?5err?$DN?$CFd?5@ 00000001800049e0     libdeclcls003.obj
 0002:00000a10       ??_C@_0CO@KBGKJPBD@stderr?3?5fflush?5failed?5?9?5err?$DN?$CFd?5@ 0000000180004a10     libdeclcls003.obj
 0002:00000a40       ??_C@_0BB@JCNMKLLK@JVMTI_ERROR_NONE@ 0000000180004a40     libdeclcls003.obj
 0002:00000a58       ??_C@_0BL@LDIMKLPH@JVMTI_ERROR_INVALID_THREAD@ 0000000180004a58     libdeclcls003.obj
 0002:00000a78       ??_C@_0CB@PJFPAIKJ@JVMTI_ERROR_INVALID_THREAD_GROU@ 0000000180004a78     libdeclcls003.obj
 0002:00000aa0       ??_C@_0BN@LLMKHMNF@JVMTI_ERROR_INVALID_PRIORITY@ 0000000180004aa0     libdeclcls003.obj
 0002:00000ac0       ??_C@_0CB@MBOFKAGB@JVMTI_ERROR_THREAD_NOT_SUSPENDE@ 0000000180004ac0     libdeclcls003.obj
 0002:00000ae8       ??_C@_0BN@FABOLPBI@JVMTI_ERROR_THREAD_SUSPENDED@ 0000000180004ae8     libdeclcls003.obj
 0002:00000b08       ??_C@_0BN@FDGNOBJM@JVMTI_ERROR_THREAD_NOT_ALIVE@ 0000000180004b08     libdeclcls003.obj
 0002:00000b28       ??_C@_0BL@GOBIFKNJ@JVMTI_ERROR_INVALID_OBJECT@ 0000000180004b28     libdeclcls003.obj
 0002:00000b48       ??_C@_0BK@FCMAJPPC@JVMTI_ERROR_INVALID_CLASS@ 0000000180004b48     libdeclcls003.obj
 0002:00000b68       ??_C@_0BP@IKLLBKEB@JVMTI_ERROR_CLASS_NOT_PREPARED@ 0000000180004b68     libdeclcls003.obj
 0002:00000b88       ??_C@_0BN@KLPPLKG@JVMTI_ERROR_INVALID_METHODID@ 0000000180004b88     libdeclcls003.obj
 0002:00000ba8       ??_C@_0BN@BCEKOKND@JVMTI_ERROR_INVALID_LOCATION@ 0000000180004ba8     libdeclcls003.obj
 0002:00000bc8       ??_C@_0BM@DFDGPME@JVMTI_ERROR_INVALID_FIELDID@ 0000000180004bc8     libdeclcls003.obj
 0002:00000be8       ??_C@_0BL@NELIEPEC@JVMTI_ERROR_NO_MORE_FRAMES@ 0000000180004be8     libdeclcls003.obj
 0002:00000c08       ??_C@_0BJ@BDBECFDM@JVMTI_ERROR_OPAQUE_FRAME@ 0000000180004c08     libdeclcls003.obj
 0002:00000c28       ??_C@_0BK@MIIFNLOB@JVMTI_ERROR_TYPE_MISMATCH@ 0000000180004c28     libdeclcls003.obj
 0002:00000c48       ??_C@_0BJ@HPCAOILC@JVMTI_ERROR_INVALID_SLOT@ 0000000180004c48     libdeclcls003.obj
 0002:00000c68       ??_C@_0BG@CHILOPNI@JVMTI_ERROR_DUPLICATE@ 0000000180004c68     libdeclcls003.obj
 0002:00000c80       ??_C@_0BG@DIEMLHKM@JVMTI_ERROR_NOT_FOUND@ 0000000180004c80     libdeclcls003.obj
 0002:00000c98       ??_C@_0BM@NHMCKHOB@JVMTI_ERROR_INVALID_MONITOR@ 0000000180004c98     libdeclcls003.obj
 0002:00000cb8       ??_C@_0BO@PPEDAJGL@JVMTI_ERROR_NOT_MONITOR_OWNER@ 0000000180004cb8     libdeclcls003.obj
 0002:00000cd8       ??_C@_0BG@FCAIPEID@JVMTI_ERROR_INTERRUPT@ 0000000180004cd8     libdeclcls003.obj
 0002:00000cf0       ??_C@_0CB@EGDBNKOI@JVMTI_ERROR_INVALID_CLASS_FORMA@ 0000000180004cf0     libdeclcls003.obj
 0002:00000d18       ??_C@_0CG@DGKOGIAL@JVMTI_ERROR_CIRCULAR_CLASS_DEFI@ 0000000180004d18     libdeclcls003.obj
 0002:00000d40       ??_C@_0BP@ICEALPKC@JVMTI_ERROR_FAILS_VERIFICATION@ 0000000180004d40     libdeclcls003.obj
 0002:00000d60       ??_C@_0DC@JDACLMIO@JVMTI_ERROR_UNSUPPORTED_REDEFIN@ 0000000180004d60     libdeclcls003.obj
 0002:00000d98       ??_C@_0DE@GKDKNOMJ@JVMTI_ERROR_UNSUPPORTED_REDEFIN@ 0000000180004d98     libdeclcls003.obj
 0002:00000dd0       ??_C@_0BO@LAFKIOG@JVMTI_ERROR_INVALID_TYPESTATE@ 0000000180004dd0     libdeclcls003.obj
 0002:00000df0       ??_C@_0DH@INDGCLLB@JVMTI_ERROR_UNSUPPORTED_REDEFIN@ 0000000180004df0     libdeclcls003.obj
 0002:00000e28       ??_C@_0DE@NHEOMMGI@JVMTI_ERROR_UNSUPPORTED_REDEFIN@ 0000000180004e28     libdeclcls003.obj
 0002:00000e60       ??_C@_0CA@EKPNJOEP@JVMTI_ERROR_UNSUPPORTED_VERSION@ 0000000180004e60     libdeclcls003.obj
 0002:00000e80       ??_C@_0BN@OFFMAHHL@JVMTI_ERROR_NAMES_DONT_MATCH@ 0000000180004e80     libdeclcls003.obj
 0002:00000ea0       ??_C@_0DN@HHBBLAKE@JVMTI_ERROR_UNSUPPORTED_REDEFIN@ 0000000180004ea0     libdeclcls003.obj
 0002:00000ee0       ??_C@_0DO@HMBGBGNA@JVMTI_ERROR_UNSUPPORTED_REDEFIN@ 0000000180004ee0     libdeclcls003.obj
 0002:00000f20       ??_C@_0BP@PBECGKHJ@JVMTI_ERROR_UNMODIFIABLE_CLASS@ 0000000180004f20     libdeclcls003.obj
 0002:00000f40       ??_C@_0BK@CANILEHF@JVMTI_ERROR_NOT_AVAILABLE@ 0000000180004f40     libdeclcls003.obj
 0002:00000f60       ??_C@_0CE@INJKMEFK@JVMTI_ERROR_MUST_POSSESS_CAPABI@ 0000000180004f60     libdeclcls003.obj
 0002:00000f88       ??_C@_0BJ@LBFPFPDM@JVMTI_ERROR_NULL_POINTER@ 0000000180004f88     libdeclcls003.obj
 0002:00000fa8       ??_C@_0BP@CHJPNNEM@JVMTI_ERROR_ABSENT_INFORMATION@ 0000000180004fa8     libdeclcls003.obj
 0002:00000fc8       ??_C@_0BP@OMFMNLC@JVMTI_ERROR_INVALID_EVENT_TYPE@ 0000000180004fc8     libdeclcls003.obj
 0002:00000fe8       ??_C@_0BN@BIBNPHHO@JVMTI_ERROR_ILLEGAL_ARGUMENT@ 0000000180004fe8     libdeclcls003.obj
 0002:00001008       ??_C@_0BK@KKNDHDCE@JVMTI_ERROR_NATIVE_METHOD@ 0000000180005008     libdeclcls003.obj
 0002:00001028       ??_C@_0BK@PMKCFHAE@JVMTI_ERROR_OUT_OF_MEMORY@ 0000000180005028     libdeclcls003.obj
 0002:00001048       ??_C@_0BK@NNJBDMNB@JVMTI_ERROR_ACCESS_DENIED@ 0000000180005048     libdeclcls003.obj
 0002:00001068       ??_C@_0BI@GHECLMNC@JVMTI_ERROR_WRONG_PHASE@ 0000000180005068     libdeclcls003.obj
 0002:00001080       ??_C@_0BF@OLIHJOII@JVMTI_ERROR_INTERNAL@ 0000000180005080     libdeclcls003.obj
 0002:00001098       ??_C@_0BO@EOHGKJHI@JVMTI_ERROR_UNATTACHED_THREAD@ 0000000180005098     libdeclcls003.obj
 0002:000010b8       ??_C@_0CA@LKHFDACL@JVMTI_ERROR_INVALID_ENVIRONMENT@ 00000001800050b8     libdeclcls003.obj
 0002:000010d8       ??_C@_0BA@MMFHLOKK@?$DMunknown?5error?$DO@ 00000001800050d8     libdeclcls003.obj
 0002:000010e8       ??_C@_0CF@CBHOKDB@throwable?5?$DN?5jni?9?$DOExceptionOccur@ 00000001800050e8     libdeclcls003.obj
 0002:00001110       ??_C@_03OFAPEBGM@?$CFs?6@  0000000180005110     libdeclcls003.obj
 0002:00001118       ??_C@_0DM@LPIGEGNJ@s?2test?2hotspot?2jtreg?2vmTestbase@ 0000000180005118     libdeclcls003.obj
 0002:00001158       ??_C@_0CC@NFCNPEPK@Exception?5in?5JNI?5call?5?$CIcleared?$CJ@ 0000000180005158     libdeclcls003.obj
 0002:00001180       ??_C@_0BJ@IBAKFIKF@jni?9?$DOExceptionDescribe?$CI?$CJ@ 0000000180005180     libdeclcls003.obj
 0002:000011a0       ??_C@_0BG@GGKALKMH@jni?9?$DOExceptionClear?$CI?$CJ@ 00000001800051a0     libdeclcls003.obj
 0002:000011b8       ??_C@_0CF@JMGFGJLJ@?$CD?5?5?5verified?5JNI?5assertion?5is?5F@ 00000001800051b8     libdeclcls003.obj
 0002:000011e0       ??_C@_0CB@MLNJNCLJ@?5?5jvmti?5error?3?5code?$DN?$CFd?0?5name?$DN?$CFs@ 00000001800051e0     libdeclcls003.obj
 0002:00001208       ??_C@_0CD@OHBGDKMK@?$CD?5?5?5jvmti?5error?3?5code?$DN?$CFd?0?5name?$DN@ 0000000180005208     libdeclcls003.obj
 0002:00001230       ??_C@_0CG@JNNCGPHB@?$CD?5?5?5error?5expected?3?5code?$DN?$CFd?0?5na@ 0000000180005230     libdeclcls003.obj
 0002:00001260       ??_C@_0EB@IMGKPCGE@?$CIstr_obj?5?$DN?5jni?9?$DONewStringUTF?$CIco@ 0000000180005260     libdeclcls003.obj
 0002:000012b0       ??_C@_0EA@HFOGGBCC@s?2test?2hotspot?2jtreg?2vmTestbase@ 00000001800052b0     libdeclcls003.obj
 0002:000012f0       ??_C@_05KKCIMGE@error@     00000001800052f0     libdeclcls003.obj
 0002:00001300       ??_C@_0EA@PNBCDMOA@s?2test?2hotspot?2jtreg?2vmTestbase@ 0000000180005300     libdeclcls003.obj
 0002:00001340       ??_C@_0DI@ILAHDLMP@?$CI?$CKagentThreadProc?$CJ?$CIjvmti_env?0?5a@ 0000000180005340     libdeclcls003.obj
 0002:00001378       ??_C@_0BD@KDBALNLB@JVMTI?5agent?5thread@ 0000000180005378     libdeclcls003.obj
 0002:00001390       ??_C@_0BB@NOKBFPFO@java?1lang?1Thread@ 0000000180005390     libdeclcls003.obj
 0002:000013a4       ??_C@_06FALKBLGB@?$DMinit?$DO@ 00000001800053a4     libdeclcls003.obj
 0002:000013b0       ??_C@_0BG@IKDDPPGD@?$CILjava?1lang?1String?$DL?$CJV@ 00000001800053b0     libdeclcls003.obj
 0002:000013d0       ??_C@_0EB@IFJBFEKC@?$CIthreadClass?5?$DN?5jni_env?9?$DOFindCla@ 00000001800053d0     libdeclcls003.obj
 0002:00001420       ??_C@_0GF@FGFIBKKL@?$CIthreadCtor?5?$DN?5jni_env?9?$DOGetMetho@ 0000000180005420     libdeclcls003.obj
 0002:00001488       ??_C@_0DN@NCPDJLOG@?$CIthreadName?5?$DN?5jni_env?9?$DONewStrin@ 0000000180005488     libdeclcls003.obj
 0002:000014d0       ??_C@_0FE@PFKODBGC@?$CIthreadObject?5?$DN?5jni_env?9?$DONewObj@ 00000001800054d0     libdeclcls003.obj
 0002:00001530       ??_C@_0ED@HOBAHHJI@?$CIthreadGlobalRef?5?$DN?5jni_env?9?$DONew@ 0000000180005530     libdeclcls003.obj
 0002:00001580       ??_C@_0FN@HNJJAHFC@jvmti_env?9?$DORunAgentThread?$CIagent@ 0000000180005580     libdeclcls003.obj
 0002:000015e0       ??_C@_0EA@MOJDNKDF@Debuggee?5status?5sync?5aborted?5be@ 00000001800055e0     libdeclcls003.obj
 0002:00001620       ??_C@_0EA@EEOEJAEN@status?5?$DN?5syncDebuggeeStatus?$CIjni@ 0000000180005620     libdeclcls003.obj
 0002:00001660       ??_C@_0BL@JBCFNBMB@nsk_jvmti_resetAgentData?$CI?$CJ@ 0000000180005660     libdeclcls003.obj
 0002:00001680       ??_C@_0EL@LPBEELIP@s?2test?2hotspot?2jtreg?2vmTestbase@ 0000000180005680     libdeclcls003.obj
 0002:000016d0       ??_C@_0CK@JDAMFDMJ@jvmti?9?$DOSetTag?$CIo?0?5tag?$CJ?5?$DN?$DN?5JVMTI_@ 00000001800056d0     libdeclcls003.obj
 0002:00001700       ??_C@_0CC@DAMNHKNI@Can?8t?5set?5tag?5?$CFli?5for?5object?5?$CFl@ 0000000180005700     libdeclcls003.obj
 0002:00001728       ??_C@_0DL@HAJPNKEF@jvmti?9?$DOGetObjectHashCode?$CIo?0?5?$CGha@ 0000000180005728     libdeclcls003.obj
 0002:00001768       ??_C@_0BL@JFPIEOBF@Can?8t?5get?5hash?5object?5?$CFlx?6@ 0000000180005768     libdeclcls003.obj
 0002:00001788       ??_C@_0BG@DICPHBKN@setTag?3?5?$CF08x?5?$DM?9?5?$CF?53li@ 0000000180005788     libdeclcls003.obj
 0002:000017a0       ??_C@_0DH@FCEEBDMJ@?$CIs?5?$DN?5jni?9?$DOGetStringUTFChars?$CIsIn@ 00000001800057a0     libdeclcls003.obj
 0002:000017d8       ??_C@_0BJ@OKKGHDCN@Can?8t?5get?5string?5at?5?$CF?$CDp?6@ 00000001800057d8     libdeclcls003.obj
 0002:000017f8       ??_C@_0BP@EKFLGGFJ@Can?8t?5get?5string?5at?5?$CF?$CDp?3?5null?6@ 00000001800057f8     libdeclcls003.obj
 0002:00001818       ??_C@_06ICODBHCL@?5?1?1?5?$CFs@ 0000000180005818     libdeclcls003.obj
 0002:00001820       ??_C@_0DB@KGFPLEGO@?$CIr?5?$DN?5jvmti?9?$DOGetTag?$CIo?0?5?$CGtag?$CJ?$CJ?5?$DN?$DN@ 0000000180005820     libdeclcls003.obj
 0002:00001858       ??_C@_0CO@PDAGBCGJ@Can?8t?5GetTag?5for?5object?5?$CFlx?4?5Re@ 0000000180005858     libdeclcls003.obj
 0002:00001888       ??_C@_0CH@HPEODOHC@TEST_BUG?3?5Max?4?5number?5of?5refs?5r@ 0000000180005888     libdeclcls003.obj
 0002:000018b0       ??_C@_0DI@PHFCABIM@?$CIr?5?$DN?5jvmti?9?$DOGetTag?$CIfrom?0?5?$CGtagFr@ 00000001800058b0     libdeclcls003.obj
 0002:000018e8       ??_C@_0DI@MDEGFNKD@TEST_BUG?3?5Can?8t?5GetTag?5for?5obje@ 00000001800058e8     libdeclcls003.obj
 0002:00001920       ??_C@_0DE@MLELJAHM@?$CIr?5?$DN?5jvmti?9?$DOGetTag?$CIto?0?5?$CGtagTo?$CJ?$CJ@ 0000000180005920     libdeclcls003.obj
 0002:00001954       ??_C@_03GAEACAIP@?$CI?$CJV@ 0000000180005954     libdeclcls003.obj
 0002:00001958       ??_C@_0BH@HGGPLJO@?$DO?$DO?$DO?5checking?3?5?$CFs?4?$CFs?$CFs?6@ 0000000180005958     libdeclcls003.obj
 0002:00001970       ??_C@_0BF@JHDKGOJP@?$CFs?4?$CFs?$CFs?3?5mid?5?$DN?5null?6@ 0000000180005970     libdeclcls003.obj
 0002:00001988       ??_C@_09EMDDFCNP@?$CFs?4?$CFs?$CFs?3?5@ 0000000180005988     libdeclcls003.obj
 0002:00001998       ??_C@_0DF@BMPOKPHD@?$CIGetMethodDeclaringClass?$CJ?5unexp@ 0000000180005998     libdeclcls003.obj
 0002:000019d0       ??_C@_0CP@HMGAFMHE@?$CIGetClassSignature?$CJ?5unexpected?5@ 00000001800059d0     libdeclcls003.obj
 0002:00001a00       ??_C@_0CA@DNANLNDI@?$DO?$DO?$DO?7method?5declaring?5class?3?5?$CFs?6@ 0000000180005a00     libdeclcls003.obj
 0002:00001a20       ??_C@_0CK@DANDBEON@declaring?5class?5expected?3?5?$CFs?0?5a@ 0000000180005a20     libdeclcls003.obj
 0002:00001a50       ??_C@_09OPJEJKBL@printdump@ 0000000180005a50     libdeclcls003.obj
 0002:00001a60       ??_C@_0CJ@KCDEKOCJ@Wrong?5result?5of?5a?5valid?5call?5to@ 0000000180005a60     libdeclcls003.obj
 0002:00001a90       ??_C@_0BF@LHBAMMHC@?$CI?$CJLjava?1lang?1Object?$DL@ 0000000180005a90     libdeclcls003.obj
 0002:00001aa8       ??_C@_05KFBJCHHJ@clone@    0000000180005aa8     libdeclcls003.obj
 0002:00001ab0       ??_C@_0BG@DHOOFEJE@?$CILjava?1lang?1Object?$DL?$CJZ@ 0000000180005ab0     libdeclcls003.obj
 0002:00001ac8       ??_C@_06IMBEHKAP@equals@   0000000180005ac8     libdeclcls003.obj
 0002:00001ad0       ??_C@_08LKAKBDAJ@finalize@ 0000000180005ad0     libdeclcls003.obj
 0002:00001ae0       ??_C@_0BE@IIFEGCLG@?$CI?$CJLjava?1lang?1Class?$DL@ 0000000180005ae0     libdeclcls003.obj
 0002:00001af8       ??_C@_08KFOJNDAP@getClass@ 0000000180005af8     libdeclcls003.obj
 0002:00001b04       ??_C@_03KNBKCOBB@?$CI?$CJI@ 0000000180005b04     libdeclcls003.obj
 0002:00001b08       ??_C@_08PAGJBGJL@hashCode@ 0000000180005b08     libdeclcls003.obj
 0002:00001b14       ??_C@_06LIGDCBBN@notify@   0000000180005b14     libdeclcls003.obj
 0002:00001b20       ??_C@_09OHPHDMCN@notifyAll@ 0000000180005b20     libdeclcls003.obj
 0002:00001b30       ??_C@_0BF@FOHFOJOB@?$CI?$CJLjava?1lang?1String?$DL@ 0000000180005b30     libdeclcls003.obj
 0002:00001b48       ??_C@_08JCDFGHAO@toString@ 0000000180005b48     libdeclcls003.obj
 0002:00001b54       ??_C@_04PNOAOIAG@wait@     0000000180005b54     libdeclcls003.obj
 0002:00001b5c       ??_C@_04OHLIFDMD@?$CIJ?$CJV@ 0000000180005b5c     libdeclcls003.obj
 0002:00001b64       ??_C@_05IKOAAJOF@?$CIJI?$CJV@ 0000000180005b64     libdeclcls003.obj
 0002:00001b80       ??_C@_1EC@JIJBPKFM@?$AAa?$AAp?$AAi?$AA?9?$AAm?$AAs?$AA?9?$AAw?$AAi?$AAn?$AA?9?$AAc?$AAo?$AAr?$AAe@ 0000000180005b80     MSVCRT:thread_safe_statics.obj
 0002:00001bc8       ??_C@_1BK@MGMFAEKH@?$AAk?$AAe?$AAr?$AAn?$AAe?$AAl?$AA3?$AA2?$AA?4?$AAd?$AAl?$AAl@ 0000000180005bc8     MSVCRT:thread_safe_statics.obj
 0002:00001be8       ??_C@_0BJ@JEBJOJFJ@SleepConditionVariableCS@ 0000000180005be8     MSVCRT:thread_safe_statics.obj
 0002:00001c08       ??_C@_0BJ@PGPPEPCC@WakeAllConditionVariable@ 0000000180005c08     MSVCRT:thread_safe_statics.obj
 0002:00001c28       _pDefaultRawDllMain        0000000180005c28     MSVCRT:dll_dllmain.obj
 0002:00001c28       _pRawDllMain               0000000180005c28     MSVCRT:dll_dllmain.obj
 0002:00001c30       __xmm@ffffffffffffffffffffffffffffffff 0000000180005c30     MSVCRT:utility.obj
 0002:00001c40       _load_config_used          0000000180005c40     MSVCRT:loadcfg.obj
 0002:00001e00       _tls_used                  0000000180005e00     MSVCRT:tlssup.obj
 0002:00001e28       __volatile_metadata        0000000180005e28     <linker-defined>
 0002:000021f0       __rtc_iaa                  00000001800061f0     MSVCRT:initsect.obj
 0002:000021f8       __rtc_izz                  00000001800061f8     MSVCRT:initsect.obj
 0002:00002200       __rtc_taa                  0000000180006200     MSVCRT:initsect.obj
 0002:00002208       __rtc_tzz                  0000000180006208     MSVCRT:initsect.obj
 0002:00002210       _tls_start                 0000000180006210     MSVCRT:tlssup.obj
 0002:00002214       _Init_thread_epoch         0000000180006214     MSVCRT:thread_safe_statics.obj
 0002:00002218       _tls_end                   0000000180006218     MSVCRT:tlssup.obj
 0002:000028b4       __IMPORT_DESCRIPTOR_KERNEL32 00000001800068b4     kernel32:KERNEL32.dll
 0002:000028c8       __IMPORT_DESCRIPTOR_VCRUNTIME140 00000001800068c8     vcruntime:VCRUNTIME140.dll
 0002:000028dc       __IMPORT_DESCRIPTOR_api-ms-win-crt-runtime-l1-1-0 00000001800068dc     ucrt:api-ms-win-crt-runtime-l1-1-0.dll
 0002:000028f0       __IMPORT_DESCRIPTOR_api-ms-win-crt-stdio-l1-1-0 00000001800068f0     ucrt:api-ms-win-crt-stdio-l1-1-0.dll
 0002:00002904       __IMPORT_DESCRIPTOR_api-ms-win-crt-string-l1-1-0 0000000180006904     ucrt:api-ms-win-crt-string-l1-1-0.dll
 0002:00002918       __NULL_IMPORT_DESCRIPTOR   0000000180006918     kernel32:KERNEL32.dll
 0003:00000090       _Init_global_epoch         0000000180007090     MSVCRT:thread_safe_statics.obj
 0003:000000a0       __security_cookie          00000001800070a0     MSVCRT:gs_cookie.obj
 0003:000000a8       __security_cookie_complement 00000001800070a8     MSVCRT:gs_cookie.obj
 0003:000000b0       __scrt_native_dllmain_reason 00000001800070b0     MSVCRT:utility.obj
 0003:000000b8       __isa_available            00000001800070b8     MSVCRT:cpu_disp.obj
 0003:000000bc       __isa_enabled              00000001800070bc     MSVCRT:cpu_disp.obj
 0003:000000c0       __memset_fast_string_threshold 00000001800070c0     MSVCRT:cpu_disp.obj
 0003:000000c8       __memset_nt_threshold      00000001800070c8     MSVCRT:cpu_disp.obj
 0003:000000d0       __scrt_ucrt_dll_is_in_use  00000001800070d0     MSVCRT:ucrt_stubs.obj
 0003:000000e0       g_wrongHeapCallbacks       00000001800070e0     libdeclcls003.obj
 0003:00000160       g_szTagInfo                0000000180007160     libdeclcls003.obj
 0003:000020a0       g_tagFlags                 00000001800090a0     libdeclcls003.obj
 0003:00002488       g_refsToVerifyCnt          0000000180009488     libdeclcls003.obj
 0003:0000248c       g_fakeUserData             000000018000948c     libdeclcls003.obj
 0003:00002490       g_tagVisitCount            0000000180009490     libdeclcls003.obj
 0003:00003430       g_refsToVerify             000000018000a430     libdeclcls003.obj
 0003:0001ab30       g_userDataError            0000000180021b30     libdeclcls003.obj
 0003:0001acd0       ?_OptionsStorage@?1??__local_stdio_printf_options@@9@4_KA 0000000180021cd0     libdeclcls003.obj
 0003:0001b298       _tls_index                 0000000180022298     MSVCRT:tlssup.obj
 0003:0001b2a0       __scrt_current_native_startup_state 00000001800222a0     MSVCRT:utility.obj
 0003:0001b2a8       __scrt_native_startup_lock 00000001800222a8     MSVCRT:utility.obj
 0003:0001b2e8       __scrt_debugger_hook_flag  00000001800222e8     MSVCRT:utility_desktop.obj
 0003:0001b2f0       ?__type_info_root_node@@3U__type_info_node@@A 00000001800222f0     MSVCRT:tncleanup.obj
 0003:0001b300       ?_OptionsStorage@?1??__local_stdio_scanf_options@@9@4_KA 0000000180022300     MSVCRT:default_local_stdio_options.obj
 0003:0001b308       __favor                    0000000180022308     MSVCRT:cpu_disp.obj
 0003:0001b310       __dyn_tls_init_callback    0000000180022310     <common>

 entry point at        0001:00002300

 Static symbols

 0000:fffdb000       .debug$S                   0000000180000000     declcls003.exp
 0000:fffdb000       .debug$S                   0000000180000000     vcruntime:VCRUNTIME140.dll
 0000:fffdb000       .debug$S                   0000000180000000     vcruntime:VCRUNTIME140.dll
 0000:fffdb000       .debug$S                   0000000180000000     vcruntime:VCRUNTIME140.dll
 0000:fffdb000       .debug$S                   0000000180000000     vcruntime:VCRUNTIME140.dll
 0000:fffdb000       .debug$S                   0000000180000000     vcruntime:VCRUNTIME140.dll
 0000:fffdb000       .debug$S                   0000000180000000     vcruntime:VCRUNTIME140.dll
 0000:fffdb000       .debug$S                   0000000180000000     vcruntime:VCRUNTIME140.dll
 0000:fffdb000       .debug$S                   0000000180000000     ucrt:api-ms-win-crt-convert-l1-1-0.dll
 0002:ffffc000       .idata$6                   0000000180000000     ucrt:api-ms-win-crt-convert-l1-1-0.dll
 0000:fffdb000       .debug$S                   0000000180000000     ucrt:api-ms-win-crt-heap-l1-1-0.dll
 0000:fffdb000       .debug$S                   0000000180000000     ucrt:api-ms-win-crt-heap-l1-1-0.dll
 0000:fffdb000       .debug$S                   0000000180000000     ucrt:api-ms-win-crt-heap-l1-1-0.dll
 0000:fffdb000       .debug$S                   0000000180000000     ucrt:api-ms-win-crt-heap-l1-1-0.dll
 0002:ffffc000       .idata$6                   0000000180000000     ucrt:api-ms-win-crt-heap-l1-1-0.dll
 0000:fffdb000       .debug$S                   0000000180000000     ucrt:api-ms-win-crt-runtime-l1-1-0.dll
 0000:fffdb000       .debug$S                   0000000180000000     ucrt:api-ms-win-crt-runtime-l1-1-0.dll
 0000:fffdb000       .debug$S                   0000000180000000     ucrt:api-ms-win-crt-runtime-l1-1-0.dll
 0000:fffdb000       .debug$S                   0000000180000000     ucrt:api-ms-win-crt-runtime-l1-1-0.dll
 0000:fffdb000       .debug$S                   0000000180000000     ucrt:api-ms-win-crt-runtime-l1-1-0.dll
 0000:fffdb000       .debug$S                   0000000180000000     ucrt:api-ms-win-crt-runtime-l1-1-0.dll
 0000:fffdb000       .debug$S                   0000000180000000     ucrt:api-ms-win-crt-runtime-l1-1-0.dll
 0000:fffdb000       .debug$S                   0000000180000000     ucrt:api-ms-win-crt-runtime-l1-1-0.dll
 0000:fffdb000       .debug$S                   0000000180000000     ucrt:api-ms-win-crt-runtime-l1-1-0.dll
 0000:fffdb000       .debug$S                   0000000180000000     ucrt:api-ms-win-crt-runtime-l1-1-0.dll
 0000:fffdb000       .debug$S                   0000000180000000     ucrt:api-ms-win-crt-runtime-l1-1-0.dll
 0000:fffdb000       .debug$S                   0000000180000000     ucrt:api-ms-win-crt-runtime-l1-1-0.dll
 0000:fffdb000       .debug$S                   0000000180000000     ucrt:api-ms-win-crt-runtime-l1-1-0.dll
 0000:fffdb000       .debug$S                   0000000180000000     ucrt:api-ms-win-crt-runtime-l1-1-0.dll
 0000:fffdb000       .debug$S                   0000000180000000     ucrt:api-ms-win-crt-runtime-l1-1-0.dll
 0000:fffdb000       .debug$S                   0000000180000000     ucrt:api-ms-win-crt-runtime-l1-1-0.dll
 0000:fffdb000       .debug$S                   0000000180000000     ucrt:api-ms-win-crt-stdio-l1-1-0.dll
 0000:fffdb000       .debug$S                   0000000180000000     ucrt:api-ms-win-crt-stdio-l1-1-0.dll
 0000:fffdb000       .debug$S                   0000000180000000     ucrt:api-ms-win-crt-stdio-l1-1-0.dll
 0000:fffdb000       .debug$S                   0000000180000000     ucrt:api-ms-win-crt-stdio-l1-1-0.dll
 0000:fffdb000       .debug$S                   0000000180000000     ucrt:api-ms-win-crt-stdio-l1-1-0.dll
 0000:fffdb000       .debug$S                   0000000180000000     ucrt:api-ms-win-crt-stdio-l1-1-0.dll
 0000:fffdb000       .debug$S                   0000000180000000     ucrt:api-ms-win-crt-stdio-l1-1-0.dll
 0000:fffdb000       .debug$S                   0000000180000000     ucrt:api-ms-win-crt-stdio-l1-1-0.dll
 0000:fffdb000       .debug$S                   0000000180000000     ucrt:api-ms-win-crt-stdio-l1-1-0.dll
 0000:fffdb000       .debug$S                   0000000180000000     ucrt:api-ms-win-crt-stdio-l1-1-0.dll
 0000:fffdb000       .debug$S                   0000000180000000     ucrt:api-ms-win-crt-string-l1-1-0.dll
 0000:fffdb000       .debug$S                   0000000180000000     ucrt:api-ms-win-crt-string-l1-1-0.dll
 0000:fffdb000       .debug$S                   0000000180000000     ucrt:api-ms-win-crt-string-l1-1-0.dll
 0000:fffdb000       .debug$S                   0000000180000000     ucrt:api-ms-win-crt-string-l1-1-0.dll
 0000:fffdb000       .debug$S                   0000000180000000     ucrt:api-ms-win-crt-string-l1-1-0.dll
 0000:fffdb000       .debug$S                   0000000180000000     ucrt:api-ms-win-crt-string-l1-1-0.dll
 0000:fffdb000       .debug$S                   0000000180000000     ucrt:api-ms-win-crt-string-l1-1-0.dll
 0000:fffdb000       .debug$S                   0000000180000000     ucrt:api-ms-win-crt-string-l1-1-0.dll
 0000:fffdb000       .debug$S                   0000000180000000     kernel32:KERNEL32.dll
 0000:fffdb000       .debug$S                   0000000180000000     kernel32:KERNEL32.dll
 0000:fffdb000       .debug$S                   0000000180000000     kernel32:KERNEL32.dll
 0000:fffdb000       .debug$S                   0000000180000000     kernel32:KERNEL32.dll
 0000:fffdb000       .debug$S                   0000000180000000     kernel32:KERNEL32.dll
 0000:fffdb000       .debug$S                   0000000180000000     kernel32:KERNEL32.dll
 0000:fffdb000       .debug$S                   0000000180000000     kernel32:KERNEL32.dll
 0000:fffdb000       .debug$S                   0000000180000000     kernel32:KERNEL32.dll
 0000:fffdb000       .debug$S                   0000000180000000     kernel32:KERNEL32.dll
 0000:fffdb000       .debug$S                   0000000180000000     kernel32:KERNEL32.dll
 0000:fffdb000       .debug$S                   0000000180000000     kernel32:KERNEL32.dll
 0000:fffdb000       .debug$S                   0000000180000000     kernel32:KERNEL32.dll
 0000:fffdb000       .debug$S                   0000000180000000     kernel32:KERNEL32.dll
 0000:fffdb000       .debug$S                   0000000180000000     kernel32:KERNEL32.dll
 0000:fffdb000       .debug$S                   0000000180000000     kernel32:KERNEL32.dll
 0000:fffdb000       .debug$S                   0000000180000000     kernel32:KERNEL32.dll
 0000:fffdb000       .debug$S                   0000000180000000     kernel32:KERNEL32.dll
 0000:fffdb000       .debug$S                   0000000180000000     kernel32:KERNEL32.dll
 0000:fffdb000       .debug$S                   0000000180000000     kernel32:KERNEL32.dll
 0000:fffdb000       .debug$S                   0000000180000000     kernel32:KERNEL32.dll
 0000:fffdb000       .debug$S                   0000000180000000     kernel32:KERNEL32.dll
 0000:fffdb000       .debug$S                   0000000180000000     kernel32:KERNEL32.dll
 0000:fffdb000       .debug$S                   0000000180000000     kernel32:KERNEL32.dll
 0000:fffdb000       .debug$S                   0000000180000000     kernel32:KERNEL32.dll
 0000:fffdb000       .debug$S                   0000000180000000     kernel32:KERNEL32.dll
 0000:fffdb000       .debug$S                   0000000180000000     kernel32:KERNEL32.dll
 0000:fffdb000       .debug$S                   0000000180000000     kernel32:KERNEL32.dll
 0000:fffdb000       .debug$S                   0000000180000000     kernel32:KERNEL32.dll
 0001:00000e0c       addRefToVerify             0000000180001e0c f   libdeclcls003.obj
 0001:00000e80       agentThreadWrapper         0000000180001e80 f   libdeclcls003.obj
 0001:000011e0       file_basename              00000001800021e0 f   libdeclcls003.obj
 0001:00001808       startAgentThreadWrapper    0000000180002808 f   libdeclcls003.obj
 0001:00001b34       syncDebuggeeStatus         0000000180002b34 f   libdeclcls003.obj
 0001:00001dbc       capture_previous_context   0000000180002dbc f   MSVCRT:gs_report.obj
 0001:00001e30       ?__scrt_initialize_thread_safe_statics@@YAHXZ 0000000180002e30 f   MSVCRT:thread_safe_statics.obj
 0001:00001f00       ?__scrt_uninitialize_thread_safe_statics@@YAXXZ 0000000180002f00 f   MSVCRT:thread_safe_statics.obj
 0001:00001fb0       $$000000                   0000000180002fb0     MSVCRT:amdsecgs.obj
 0001:00001fe0       ?dllmain_crt_dispatch@@YAHQEAUHINSTANCE__@@KQEAX@Z 0000000180002fe0 f   MSVCRT:dll_dllmain.obj
 0001:00002030       ?dllmain_crt_process_attach@@YAHQEAUHINSTANCE__@@QEAX@Z 0000000180003030 f   MSVCRT:dll_dllmain.obj
 0001:00002148       ?dllmain_crt_process_detach@@YAH_N@Z 0000000180003148 f   MSVCRT:dll_dllmain.obj
 0001:000021cc       ?dllmain_dispatch@@YAHQEAUHINSTANCE__@@KQEAX@Z 00000001800031cc f   MSVCRT:dll_dllmain.obj
 0001:00002be0       $$000000                   0000000180003be0     MSVCRT:guard_dispatch.obj
 0001:00002c00       $$000000                   0000000180003c00     MSVCRT:guard_xfg_dispatch.obj
 0001:00002c16       ?fin$0@?0??dllmain_crt_process_attach@@YAHQEAUHINSTANCE__@@QEAX@Z@4HA 0000000180003c16 f   MSVCRT:dll_dllmain.obj
 0001:00002c2d       ?fin$0@?0??dllmain_crt_process_detach@@YAH_N@Z@4HA 0000000180003c2d f   MSVCRT:dll_dllmain.obj
 0001:00002c46       ?fin$1@?0??dllmain_crt_process_detach@@YAH_N@Z@4HA 0000000180003c46 f   MSVCRT:dll_dllmain.obj
 0001:00002c5a       ?filt$0@?0??dllmain_dispatch@@YAHQEAUHINSTANCE__@@KQEAX@Z@4HA 0000000180003c5a f   MSVCRT:dll_dllmain.obj
 0001:00002c90       __scrt_is_nonwritable_in_current_image$filt$0 0000000180003c90 f   MSVCRT:utility.obj
 0002:000001e8       ?__scrt_initialize_tss_var@@3P6AHXZEA 00000001800041e8     MSVCRT:thread_safe_statics.obj
 0002:00000310       ?opcLengths@@3QBEB         0000000180004310     libdeclcls003.obj
 0002:00001b70       GS_ExceptionPointers       0000000180005b70     MSVCRT:gs_report.obj
 0002:00002220       $unwind$fprintf            0000000180006220     libdeclcls003.obj
 0002:0000222c       $unwind$printf             000000018000622c     libdeclcls003.obj
 0002:00002238       $unwind$?NewObject@JNIEnv_@@QEAAPEAV_jobject@@PEAV_jclass@@PEAU_jmethodID@@ZZ 0000000180006238     libdeclcls003.obj
 0002:00002238       $unwind$nsk_lcomplain      0000000180006238     libdeclcls003.obj
 0002:00002238       $unwind$nsk_ldisplay       0000000180006238     libdeclcls003.obj
 0002:00002240       $unwind$nsk_lvdisplay      0000000180006240     libdeclcls003.obj
 0002:00002240       $unwind$_RTC_Initialize    0000000180006240     MSVCRT:initsect.obj
 0002:00002240       $unwind$_RTC_Terminate     0000000180006240     MSVCRT:initsect.obj
 0002:00002240       $unwind$?__scrt_initialize_thread_safe_statics@@YAHXZ 0000000180006240     MSVCRT:thread_safe_statics.obj
 0002:0000224c       $unwind$nsk_lvcomplain     000000018000624c     libdeclcls003.obj
 0002:00002264       $unwind$nsk_ltrace         0000000180006264     libdeclcls003.obj
 0002:00002264       $unwind$__report_gsfailure 0000000180006264     MSVCRT:gs_report.obj
 0002:0000226c       $unwind$Agent_Initialize   000000018000626c     libdeclcls003.obj
 0002:0000226c       $unwind$nsk_lvtrace        000000018000626c     libdeclcls003.obj
 0002:0000226c       $unwind$__raise_securityfailure 000000018000626c     MSVCRT:gs_report.obj
 0002:0000226c       $unwind$__scrt_initialize_crt 000000018000626c     MSVCRT:utility.obj
 0002:0000226c       $unwind$__scrt_initialize_onexit_tables 000000018000626c     MSVCRT:utility.obj
 0002:0000226c       $unwind$__scrt_release_startup_lock 000000018000626c     MSVCRT:utility.obj
 0002:0000226c       $unwind$__scrt_uninitialize_crt 000000018000626c     MSVCRT:utility.obj
 0002:0000226c       $unwind$_onexit            000000018000626c     MSVCRT:utility.obj
 0002:00002274       $unwind$nsk_lverify        0000000180006274     libdeclcls003.obj
 0002:00002284       $unwind$nsk_vprintf        0000000180006284     libdeclcls003.obj
 0002:00002294       $unwind$nsk_printf         0000000180006294     libdeclcls003.obj
 0002:0000229c       $unwind$?nsk_jni_lverify@@YAHHPEAUJNIEnv_@@HQEBDH1ZZ 000000018000629c     libdeclcls003.obj
 0002:000022b0       $unwind$?nsk_jni_check_exception@@YAHPEAUJNIEnv_@@QEBDH@Z 00000001800062b0     libdeclcls003.obj
 0002:000022cc       $unwind$Java_nsk_jvmti_unit_FollowReferences_FollowRefObjects_resetTags 00000001800062cc     libdeclcls003.obj
 0002:000022cc       $unwind$addRefToVerify     00000001800062cc     libdeclcls003.obj
 0002:000022cc       $unwind$nsk_jvmti_resetAgentData 00000001800062cc     libdeclcls003.obj
 0002:000022cc       $unwind$__scrt_initialize_default_local_stdio_options 00000001800062cc     MSVCRT:default_local_stdio_options.obj
 0002:000022cc       $unwind$?dllmain_crt_dispatch@@YAHQEAUHINSTANCE__@@KQEAX@Z 00000001800062cc     MSVCRT:dll_dllmain.obj
 0002:000022cc       $unwind$DllMain            00000001800062cc     MSVCRT:dll_dllmain_stub.obj
 0002:000022cc       $unwind$__GSHandlerCheck   00000001800062cc     MSVCRT:gshandler.obj
 0002:000022cc       $unwind$?__scrt_uninitialize_thread_safe_statics@@YAXXZ 00000001800062cc     MSVCRT:thread_safe_statics.obj
 0002:000022cc       $unwind$__scrt_acquire_startup_lock 00000001800062cc     MSVCRT:utility.obj
 0002:000022cc       $unwind$__scrt_dllmain_after_initialize_c 00000001800062cc     MSVCRT:utility.obj
 0002:000022cc       $unwind$__scrt_dllmain_before_initialize_c 00000001800062cc     MSVCRT:utility.obj
 0002:000022cc       $unwind$__scrt_dllmain_crt_thread_attach 00000001800062cc     MSVCRT:utility.obj
 0002:000022cc       $unwind$__scrt_dllmain_crt_thread_detach 00000001800062cc     MSVCRT:utility.obj
 0002:000022cc       $unwind$__scrt_dllmain_uninitialize_c 00000001800062cc     MSVCRT:utility.obj
 0002:000022cc       $unwind$__scrt_dllmain_uninitialize_critical 00000001800062cc     MSVCRT:utility.obj
 0002:000022cc       $unwind$atexit             00000001800062cc     MSVCRT:utility.obj
 0002:000022d4       $unwind$nsk_jvmti_lverify  00000001800062d4     libdeclcls003.obj
 0002:000022e8       $unwind$exitOnError        00000001800062e8     libdeclcls003.obj
 0002:000022f8       $unwind$Java_nsk_share_jvmti_ArgumentHandler_getAgentOptionsString 00000001800062f8     libdeclcls003.obj
 0002:0000230c       $unwind$Java_nsk_jvmti_unit_FollowReferences_FollowRefObjects_getTag 000000018000630c     libdeclcls003.obj
 0002:0000230c       $unwind$Java_nsk_share_jvmti_DebugeeClass_checkStatus 000000018000630c     libdeclcls003.obj
 0002:0000230c       $unwind$agentThreadWrapper 000000018000630c     libdeclcls003.obj
 0002:0000231c       $unwind$startAgentThreadWrapper 000000018000631c     libdeclcls003.obj
 0002:00002338       $unwind$syncDebuggeeStatus 0000000180006338     libdeclcls003.obj
 0002:00002338       $unwind$__scrt_dllmain_exception_filter 0000000180006338     MSVCRT:utility.obj
 0002:0000234c       $unwind$Java_nsk_share_jvmti_DebugeeClass_resetAgentData 000000018000634c     libdeclcls003.obj
 0002:00002354       $unwind$MA_checkStatus     0000000180006354     libdeclcls003.obj
 0002:00002368       $unwind$Java_nsk_jvmti_unit_FollowReferences_FollowRefObjects_setTag 0000000180006368     libdeclcls003.obj
 0002:00002380       $unwind$Java_nsk_jvmti_unit_FollowReferences_FollowRefObjects_addRefToVerify 0000000180006380     libdeclcls003.obj
 0002:0000239c       $unwind$do_check           000000018000639c     libdeclcls003.obj
 0002:000023b0       $unwind$Java_nsk_jvmti_GetMethodDeclaringClass_declcls003_check 00000001800063b0     libdeclcls003.obj
 0002:000023b0       $unwind$_DllMainCRTStartup 00000001800063b0     MSVCRT:dll_dllmain.obj
 0002:000023c0       $unwind$capture_previous_context 00000001800063c0     MSVCRT:gs_report.obj
 0002:000023cc       $unwind$__GSHandlerCheckCommon 00000001800063cc     MSVCRT:gshandler.obj
 0002:000023d8       $xdatasym                  00000001800063d8     MSVCRT:amdsecgs.obj
 0002:000023dc       $unwind$?dllmain_crt_process_attach@@YAHQEAUHINSTANCE__@@QEAX@Z 00000001800063dc     MSVCRT:dll_dllmain.obj
 0002:00002418       $unwind$?fin$0@?0??dllmain_crt_process_attach@@YAHQEAUHINSTANCE__@@QEAX@Z@4HA 0000000180006418     MSVCRT:dll_dllmain.obj
 0002:00002418       $unwind$?fin$0@?0??dllmain_crt_process_detach@@YAH_N@Z@4HA 0000000180006418     MSVCRT:dll_dllmain.obj
 0002:00002418       $unwind$?fin$1@?0??dllmain_crt_process_detach@@YAH_N@Z@4HA 0000000180006418     MSVCRT:dll_dllmain.obj
 0002:00002420       $unwind$?dllmain_crt_process_detach@@YAH_N@Z 0000000180006420     MSVCRT:dll_dllmain.obj
 0002:00002474       $unwind$?dllmain_dispatch@@YAHQEAUHINSTANCE__@@KQEAX@Z 0000000180006474     MSVCRT:dll_dllmain.obj
 0002:0000249c       $unwind$?filt$0@?0??dllmain_dispatch@@YAHQEAUHINSTANCE__@@KQEAX@Z@4HA 000000018000649c     MSVCRT:dll_dllmain.obj
 0002:000024a4       $unwind$__scrt_is_nonwritable_in_current_image 00000001800064a4     MSVCRT:utility.obj
 0002:000024c4       $unwind$__scrt_is_nonwritable_in_current_image$filt$0 00000001800064c4     MSVCRT:utility.obj
 0002:000024cc       $unwind$__scrt_fastfail    00000001800064cc     MSVCRT:utility_desktop.obj
 0002:000024dc       $unwind$__security_init_cookie 00000001800064dc     MSVCRT:gs_support.obj
 0002:000024e8       $unwind$__isa_available_init 00000001800064e8     MSVCRT:cpu_disp.obj
 0002:000024f8       $xdatasym                  00000001800064f8     MSVCRT:guard_dispatch.obj
 0002:00002500       $xdatasym                  0000000180006500     MSVCRT:guard_xfg_dispatch.obj
 0002:00002510       .edata                     0000000180006510     declcls003.exp
 0002:00002538       rgpv                       0000000180006538     declcls003.exp
 0002:00002574       rgszName                   0000000180006574     declcls003.exp
 0002:000025b0       rgwOrd                     00000001800065b0     declcls003.exp
 0002:000025ce       szName                     00000001800065ce     declcls003.exp
 0002:000025dd       $N00001                    00000001800065dd     declcls003.exp
 0002:000025ec       $N00002                    00000001800065ec     declcls003.exp
 0002:000025f9       $N00003                    00000001800065f9     declcls003.exp
 0002:00002631       $N00004                    0000000180006631     declcls003.exp
 0002:00002676       $N00005                    0000000180006676     declcls003.exp
 0002:000026b3       $N00006                    00000001800066b3     declcls003.exp
 0002:000026fb       $N00007                    00000001800066fb     declcls003.exp
 0002:0000273b       $N00008                    000000018000673b     declcls003.exp
 0002:00002778       $N00009                    0000000180006778     declcls003.exp
 0002:000027b3       $N00010                    00000001800067b3     declcls003.exp
 0002:000027e1       $N00011                    00000001800067e1     declcls003.exp
 0002:00002812       $N00012                    0000000180006812     declcls003.exp
 0002:00002841       $N00013                    0000000180006841     declcls003.exp
 0002:00002870       $N00014                    0000000180006870     declcls003.exp
 0002:000028a5       $N00015                    00000001800068a5     declcls003.exp
 0002:00002cb2       .idata$6                   0000000180006cb2     kernel32:KERNEL32.dll
 0002:00002d16       .idata$6                   0000000180006d16     vcruntime:VCRUNTIME140.dll
 0002:00002e82       .idata$6                   0000000180006e82     ucrt:api-ms-win-crt-runtime-l1-1-0.dll
 0002:00002ea4       .idata$6                   0000000180006ea4     ucrt:api-ms-win-crt-stdio-l1-1-0.dll
 0002:00002ec4       .idata$6                   0000000180006ec4     ucrt:api-ms-win-crt-string-l1-1-0.dll
 0003:00000000       ?codeAttributeName@@3PEBDEB 0000000180007000     libdeclcls003.obj
 0003:00000008       ?lineNumberAttributeName@@3PEBDEB 0000000180007008     libdeclcls003.obj
 0003:00000010       ?localVarAttributeName@@3PEBDEB 0000000180007010     libdeclcls003.obj
 0003:00000018       ?localVarTypeAttributeName@@3PEBDEB 0000000180007018     libdeclcls003.obj
 0003:00000020       ?stackMapAttributeName@@3PEBDEB 0000000180007020     libdeclcls003.obj
 0003:00000028       ?callBytes@@3PAEA          0000000180007028     libdeclcls003.obj
 0003:0000002c       ?allocBytes@@3PAEA         000000018000702c     libdeclcls003.obj
 0003:00000030       exp_class_sig              0000000180007030     libdeclcls003.obj
 0003:00000040       arr_sigs                   0000000180007040     libdeclcls003.obj
 0003:0001ab34       redefineAttempted          0000000180021b34     libdeclcls003.obj
 0003:0001ab38       nsk_context                0000000180021b38     libdeclcls003.obj
 0003:0001ab44       redefineSucceed            0000000180021b44     libdeclcls003.obj
 0003:0001ab48       agentFailed                0000000180021b48     libdeclcls003.obj
 0003:0001ab4c       currentAgentStatus         0000000180021b4c     libdeclcls003.obj
 0003:0001ab50       context                    0000000180021b50     libdeclcls003.obj
 0003:0001ac08       agentThread                0000000180021c08     libdeclcls003.obj
 0003:0001ac10       agentThreadProc            0000000180021c10     libdeclcls003.obj
 0003:0001ac18       agentThreadArg             0000000180021c18     libdeclcls003.obj
 0003:0001ac20       agent_data                 0000000180021c20     libdeclcls003.obj
 0003:0001ac30       jvmti_env                  0000000180021c30     libdeclcls003.obj
 0003:0001ac38       jvm                        0000000180021c38     libdeclcls003.obj
 0003:0001ac40       jni_env                    0000000180021c40     libdeclcls003.obj
 0003:0001ac48       checkStatus_func           0000000180021c48     libdeclcls003.obj
 0003:0001ac50       ?codeAttributeIndex@@3GA   0000000180021c50     libdeclcls003.obj
 0003:0001ac52       printdump                  0000000180021c52     libdeclcls003.obj
 0003:0001ac54       ?lineNumberAttributeIndex@@3GA 0000000180021c54     libdeclcls003.obj
 0003:0001ac58       ?localVarAttributeIndex@@3GA 0000000180021c58     libdeclcls003.obj
 0003:0001ac5c       ?localVarTypeAttributeIndex@@3GA 0000000180021c5c     libdeclcls003.obj
 0003:0001ac60       ?stackMapAttributeIndex@@3GA 0000000180021c60     libdeclcls003.obj
 0003:0001ac64       ?stackFrameOffset@@3GA     0000000180021c64     libdeclcls003.obj
 0003:0001ac68       ?mode@@3HA                 0000000180021c68     libdeclcls003.obj
 0003:0001ac6c       ?constantPoolSize@@3GA     0000000180021c6c     libdeclcls003.obj
 0003:0001ac70       ?orig@@3PEBEEB             0000000180021c70     libdeclcls003.obj
 0003:0001ac78       ?gen@@3PEAEEA              0000000180021c78     libdeclcls003.obj
 0003:0001ac80       ?inputPos@@3PEAEEA         0000000180021c80     libdeclcls003.obj
 0003:0001ac88       ?endPos@@3PEBEEB           0000000180021c88     libdeclcls003.obj
 0003:0001ac90       ?genPos@@3PEAEEA           0000000180021c90     libdeclcls003.obj
 0003:0001ac98       ?markPos@@3PEAEEA          0000000180021c98     libdeclcls003.obj
 0003:0001aca0       ?constantPool@@3PEAPEADEA  0000000180021ca0     libdeclcls003.obj
 0003:0001aca8       ?constantPoolCount@@3GA    0000000180021ca8     libdeclcls003.obj
 0003:0001acac       ?zeroBytes@@3PAEA          0000000180021cac     libdeclcls003.obj
 0003:0001acb0       ?codeLength@@3IA           0000000180021cb0     libdeclcls003.obj
 0003:0001acb4       result                     0000000180021cb4     libdeclcls003.obj
 0003:0001acb8       ?map@@3PEAIEA              0000000180021cb8     libdeclcls003.obj
 0003:0001acc0       ?widening@@3PEACEA         0000000180021cc0     libdeclcls003.obj
 0003:0001acc8       jvmti                      0000000180021cc8     libdeclcls003.obj
 0003:0001ace0       GS_ExceptionRecord         0000000180021ce0     MSVCRT:gs_report.obj
 0003:0001ad80       GS_ContextRecord           0000000180021d80     MSVCRT:gs_report.obj
 0003:0001b250       ?g_tss_cv@@3U_RTL_CONDITION_VARIABLE@@A 0000000180022250     MSVCRT:thread_safe_statics.obj
 0003:0001b258       ?g_tss_event@@3PEAXEA      0000000180022258     MSVCRT:thread_safe_statics.obj
 0003:0001b260       ?g_tss_mutex@@3U_RTL_CRITICAL_SECTION@@A 0000000180022260     MSVCRT:thread_safe_statics.obj
 0003:0001b288       ?g_sleep_condition_variable_cs@@3P6AHPEAU_RTL_CONDITION_VARIABLE@@PEAU_RTL_CRITICAL_SECTION@@K@ZEA 0000000180022288     MSVCRT:thread_safe_statics.obj
 0003:0001b290       ?g_wake_all_condition_variable@@3P6AXPEAU_RTL_CONDITION_VARIABLE@@@ZEA 0000000180022290     MSVCRT:thread_safe_statics.obj
 0003:0001b29c       ?__proc_attached@@3HA      000000018002229c     MSVCRT:dll_dllmain.obj
 0003:0001b2b0       ?is_initialized_as_dll@@3_NA 00000001800222b0     MSVCRT:utility.obj
 0003:0001b2b1       ?module_local_atexit_table_initialized@@3_NA 00000001800222b1     MSVCRT:utility.obj
 0003:0001b2b8       ?module_local_atexit_table@@3U_onexit_table_t@@A 00000001800222b8     MSVCRT:utility.obj
 0003:0001b2d0       ?module_local_at_quick_exit_table@@3U_onexit_table_t@@A 00000001800222d0     MSVCRT:utility.obj
